:082E340033302E312020200074
:082C4C00C116C11D4103150072
:061A0000E4900315F02242
:072E4C009003157401F02250
:0224C400AC0763
:1024C60074562BF8E6FF74562CF8E6FB900306F0DC
:1024D600EFC39480500D9003057401F0C374809F80
:1024E600F98009E4900305F0EF2480F9ED89F0A462
:1024F600FF900301E5F0F0A3EFF0900305E06028FC
:10250600900301E0FF3395E0FEC3EB9FFFE49EFEE0
:10251600900303F0A3EFF0C3EE64809480503AE496
:10252600900303F0A3F08031900301E0FF3395E0C0
:10253600FE74562CF8E6FD7C00EF2DFFEC3EFE9077
:102546000303F0A3EFF0D394FFEE64809480400978
:10255600900303E4F0A374FFF0900303E0FCA3E010
:10256600FDD394FFEC6480948040037FFF22AF0587
:012576002242
:02240D00A9051F
:10240F0074562BF8E6FE74562FF8E6FBEEC3947F56
:10241F0050097A01C3747F9EFE8006E4FA74812E00
:10242F00FEEEFD7C00AF017E00121491EF7807CE17
:10243F00A2E713CE13D8F8FFEA601FEBC39FFDE4AA
:10244F009EFC900331F0A3EDF0C3EC6480948050B8
:10245F0029E4900331F0A3F08020EB2FFFE43EFE40
:10246F00900331F0A3EFF0D394FFEE64809480409B
:10247F0009900331E4F0A374FFF0900331E0FEA361
:10248F00E0FF7C007D62121491900331EEF0A3EF18
:10249F00F0900331E0FEA3E0FF7D7F1214A39003C1
:1024AF0031EEF0A3EFF0E0241DF0900331E03400A3
:0424BF00F0A3E0FFA7
:0124C30022F6
:072DFF00E528FD3395E0FC1F
:042E0600ED2FFF228B
:102AF00074562DF8E6900339F0122D84EF2480FFF0
:102B0000900339E0FD7C00EF3395E0FE1214917CD8
:062B1000047DB01214A3C5
:012B1600229C
:072E53005355F8EF42552230
:0715AC007F01122D848F1C4A
:1015B300C200C3E51C950DFEE49400900333F0A331
:1015C300CEF0300D2E900333E0FEA3E0FFC3EE64B4
:1015D300809480500FE51670037516031516E516F3
:1015E3007049802BD3EF9406EE648094804039C217
:1015F3000D802E900333E0FEA3E0FFD39400EE644E
:10160300809480400FE5167003751603D5161C757C
:101613001601800DC3EF94FAEE6480947F5009D2D3
:101623000D851C0DD2008003E4F516E5094508700D
:1016330054300051300408850D59122D9A804630DC
:101643000D20E50D2406FFE433FED3E5599FEE6438
:1016530080F874809840028010E559C3950D501EA0
:101663008017E559D3950D4005122DE78017E50D39
:1016730024FAFFE559C39F5005122DF38007E4F5C3
:051683004FD220D2044B
:071688007F06122D848F1C68
:10168F00C200C3E51C9511FEE49400900333F0A350
:10169F00CEF030112E900333E0FEA3E0FFC3EE64D3
:1016AF00809480500FE51A7003751A03151AE51A06
:1016BF007049802BD3EF9406EE648094804039C23A
:1016CF0011802E900333E0FEA3E0FFD39400EE646D
:1016DF00809480400FE51A7003751A03D51A1C7594
:1016EF001A01800DC3EF94FAEE6480947F5009D2F3
:1016FF0011851C11D2008003E4F51AE50945087025
:10170F005430005130080885115D122D9A804630F3
:10171F001120E5112406FFE433FED3E55D9FEE644F
:10172F0080F874809840028010E55DC39511501EBB
:10173F008017E55DD395114005122DE78017E51150
:10174F0024FAFFE55DC39F5005122DF38007E4F5E2
:05175F004FD220D2086A
:101764007F07122D84AD077B077F031224C48F509B
:011774002252
:07218200E4FF122D848F1C05
:10218900C200C3E51C9512FEE49400900335F0A348
:10219900CEF030122E900335E0FEA3E0FFC3EE64CB
:1021A900809480500FE51B7003751B03151BE51BFD
:1021B9007049802BD3EF9406EE648094804039C235
:1021C90012802E900335E0FEA3E0FFD39400EE6465
:1021D900809480400FE51B7003751B03D51B1C758C
:1021E9001B01800DC3EF94FAEE6480947F5009D2ED
:1021F90012851C12D2008003E4F51BE5094508701D
:102209005430005130090885125E122D9A804630EB
:102219001220E5122406FFE433FED3E55E9FEE6447
:1022290080F874809840028010E55EC39512501EB4
:102239008017E55ED395124005122DE78017E51248
:1022490024FAFFE55EC39F5005122DF38007E4F5DC
:052259004FD220D20964
:0D225E00E55EC313FFE545C3132FF54522D0
:10089A00122CA3900316E0FF122DDA75CFE443F66B
:1008AA0002E5B05407F54E7F01122E537E807F0079
:1008BA008E2C8F2D8E298F2AE4FF122D848F45EFDF
:1008CA0090960093754C00F54D25E0FFE54C33FEFC
:1008DA0074002FF58274973EF583E493F54C740106
:1008EA0093F54D122D3D7508007509C81215AC75A2
:1008FA00F002E550A42400F582E5F03494F583E48F
:10090A0093F53D740193F53E122182122CF2122ABC
:10091A0095D2AFD2CA43C90490031630A6057430E3
:10092A00F080037431F01229F6302005C220122912
:10093A00F6E55520E303020EEB301703020C117F94
:06094A0004122DCD8F1CEC
:10095000C200C3E51C950EFEE49400900280F0A353
:10096000CEF0300E2E900280E0FEA3E0FFC3EE64D6
:10097000809480500FE51770037517031517E5175E
:100980007049802BD3EF9406EE648094804039C286
:100990000E802E900280E0FEA3E0FFD39400EE6470
:1009A000809480400FE5177003751703D5171C75E9
:1009B0001701800DC3EF94FAEE6480947F5009D242
:1009C0000E851C0ED2008003E4F517E5094508707A
:1009D00054300051300508850E5A122D9A80463049
:1009E0000E20E50E2406FFE433FED3E55A9FEE64A5
:1009F00080F874809840028010E55AC3950E501E0E
:100A00008017E55AD3950E4005122DE78017E50EA5
:100A100024FAFFE55AC39F5005122DF38007E4F531
:050A20004FD220D205B9
:070A25007F05122DCD8F1C8F
:100A2C00C200C3E51C950FFEE49400900280F0A375
:100A3C00CEF0300F2E900280E0FEA3E0FFC3EE64F8
:100A4C00809480500FE51870037518031518E5187D
:100A5C007049802BD3EF9406EE648094804039C2A9
:100A6C000F802E900280E0FEA3E0FFD39400EE6492
:100A7C00809480400FE5187003751803D5181C7509
:100A8C001801800DC3EF94FAEE6480947F5009D264
:100A9C000F851C0FD2008003E4F518E5094508709A
:100AAC0054300051300608850F5B122D9A80463069
:100ABC000F20E50F2406FFE433FED3E55B9FEE64C5
:100ACC0080F874809840028010E55BC3950F501E2F
:100ADC008017E55BD3950F4005122DE78017E50FC6
:100AEC0024FAFFE55BC39F5005122DF38007E4F554
:050AFC004FD220D206DC
:100B01007F07122DCDAD077B057F0412240D122D19
:100B1100FF75F002EFA42400F582E5F03490F5832F
:100B2100E493F53F740193F540D2177F06122DCD62
:020B31008F1C17
:100B3300C200C3E51C9510FEE49400900280F0A36C
:100B4300CEF030102E900280E0FEA3E0FFC3EE64EF
:100B5300809480500FE51970037519031519E51971
:100B63007049802BD3EF9406EE648094804039C2A1
:100B730010802E900280E0FEA3E0FFD39400EE6489
:100B8300809480400FE5197003751903D5191C75FE
:100B93001901800DC3EF94FAEE6480947F5009D25B
:100BA30010851C10D2008003E4F519E5094508708F
:100BB3005430005130070885105C122D9A8046305E
:100BC3001020E5102406FFE433FED3E55C9FEE64BA
:100BD30080F874809840028010E55CC39510501E25
:100BE3008017E55CD395104005122DE78017E510BB
:100BF30024FAFFE55CC39F5005122DF38007E4F54B
:050C03004FD220D207D2
:100C08007D067F05122AF08F28301803020EE1E4D2
:060C1800FF122DCD8F1C20
:100C1E00C200C3E51C950AFEE49400900280F0A386
:100C2E00CEF0300A2E900280E0FEA3E0FFC3EE6409
:100C3E00809480500FE51370037513031513E5139D
:100C4E007049802BD3EF9406EE648094804039C2B5
:100C5E000A802E900280E0FEA3E0FFD39400EE64A3
:100C6E00809480400FE5137003751303D5131C7524
:100C7E001301800DC3EF94FAEE6480947F5009D275
:100C8E000A851C0AD2008003E4F513E509450870B5
:100C9E0054300051300108850A56122D9A80463084
:100CAE000A20E50A2406FFE433FED3E5569FEE64E0
:100CBE0080F874809840028010E556C3950A501E45
:100CCE008017E556D3950A4005122DE78017E50AE1
:100CDE0024FAFFE556C39F5005122DF38007E4F565
:050CEE004FD220D201ED
:070CF3007F01122DCD8F1CC3
:100CFA00C200C3E51C950BFEE49400900280F0A3A9
:100D0A00CEF0300B2E900280E0FEA3E0FFC3EE642B
:100D1A00809480500FE51470037514031514E514BC
:100D2A007049802BD3EF9406EE648094804039C2D8
:100D3A000B802E900280E0FEA3E0FFD39400EE64C5
:100D4A00809480400FE5147003751403D5141C7544
:100D5A001401800DC3EF94FAEE6480947F5009D297
:100D6A000B851C0BD2008003E4F514E509450870D5
:100D7A0054300051300208850B57122D9A804630A4
:100D8A000B20E50B2406FFE433FED3E5579FEE6400
:100D9A0080F874809840028010E557C3950B501E66
:100DAA008017E557D3950B4005122DE78017E50B01
:100DBA0024FAFFE557C39F5005122DF38007E4F587
:050DCA004FD220D2020F
:100DCF007F03122DCDAD077B01E4FF12240DE52B20
:100DDF00122E0175F002EFA42400F582E5F0349095
:100DEF00F583E493F541740193F542D2187F021213
:040DFF002DCD8F1C4B
:100E0300C200C3E51C950CFEE49400900280F0A39D
:100E1300CEF0300C2E900280E0FEA3E0FFC3EE6420
:100E2300809480500FE51570037515031515E515AE
:100E33007049802BD3EF9406EE648094804039C2CE
:100E43000C802E900280E0FEA3E0FFD39400EE64BA
:100E5300809480400FE5157003751503D5151C7537
:100E63001501800DC3EF94FAEE6480947F5009D28C
:100E73000C851C0CD2008003E4F515E509450870C8
:100E830054300051300308850C58122D9A80463097
:100E93000C20E50C2406FFE433FED3E5589FEE64F3
:100EA30080F874809840028010E558C3950C501E5A
:100EB3008017E558D3950C4005122DE78017E50CF4
:100EC30024FAFFE558C39F5005122DF38007E4F57C
:050ED3004FD220D20304
:100ED8007D027F04122AF08F2BE4F530F531F5A05E
:030EE80002109A5B
:0D0EEB001215AC1221827F06122DCD8F1C36
:100EF800C200C3E51C9510FEE49400900282F0A3A2
:100F0800CEF030102E900282E0FEA3E0FFC3EE6424
:100F1800809480500FE51970037519031519E519A8
:100F28007049802BD3EF9406EE648094804039C2D8
:100F380010802E900282E0FEA3E0FFD39400EE64BE
:100F4800809480400FE5197003751903D5191C7535
:100F58001901800DC3EF94FAEE6480947F5009D292
:100F680010851C10D2008003E4F519E509450870C6
:100F78005430005130070885105C122D9A80463095
:100F88001020E5102406FFE433FED3E55C9FEE64F1
:100F980080F874809840028010E55CC39510501E5C
:100FA8008017E55CD395104005122DE78017E510F2
:100FB80024FAFFE55CC39F5005122DF38007E4F582
:050FC8004FD220D2070A
:100FCD007D067F05122AF08F28E55530E21075F069
:100FDD0002E545A42432F582E5F03497801AE54503
:100FED0090960093753400F53525E0FFE53433FE1A
:100FFD0074002FF58274973EF583E493FF7401938B
:10100D00900280CFF0A3EFF0C2A9900280E0F54CE2
:10101D00A3E0F54D75F002E550A42400F582E5F04E
:10102D003494F583E493F53D740193F53EC3E53DAA
:10103D00648094804004D21B800DC21BC3E4953E96
:10104D00F53EE4953DF53D20171FAF51122DFF756F
:10105D00F002EFA42400F582E5F03492F583E493D9
:10106D00F53F740193F540D21720181FAF52122D82
:10107D00FF75F002EFA42400F582E5F03492F583BC
:0D108D00E493F541740193F542D218D2A905
:10109A00E527605D24FE604D24FE60282403704B22
:1010AA00301615A21CB3921C301C06C226D21E8012
:1010BA003AC21E122D3D8033E49002B2F0122E7312
:1010CA00C21E8027122D9AE55530E0047F02801057
:1010DA00E55530E1047F048007E55530E20A7F01D7
:1010EA00122E538003635508122D9A1229F6E4F53D
:1010FA0027301D0E900315E07006A3E0FF122BCDDA
:10110A00C21D7B017A027964122AC4EF70030209B4
:10111A0033900266E0121505118F0411D60511519C
:10112A001411411611471711561A11781B11831DF4
:10113A0011891E00001226D21CD21E8004C21CC2B3
:10114A001E1229F6021226D2160212267B017A02F2
:10115A007964900274EBF0A3EAF0A3E9F012141791
:10116A00FE900316E0FF6E600302122680059003CC
:10117A0016E0FF122BEE021226122E4C0212261233
:10118A001A000212267B017A027964900277EBF048
:10119A00A3EAF0A3E9F0900003121430FF900316BB
:1011AA00E06F7078301C6D90027704F0A3EAF0A328
:1011BA00E9F0900005121430FF900006121430FD79
:1011CA00900004121430FB12257780487B017A02C2
:1011DA007964900277EBF0A3EAF0A3E9F0900003B8
:1011EA00121430FF900316E06F7031301C26900203
:1011FA007704F0A3EAF0A3E9F0900005121430FF97
:10120A00900006121430FD900004121430FB1223D1
:10121A0054122A95900316E0FF122C0F201C030289
:10122A00110C900266E014604814602224FB606A84
:10123A001470030212EF24F9600302110C90027D6C
:10124A007401F0A37402F0A37464F002110C121A70
:10125A00217B017A027964900274EBF0A3EAF0A38D
:10126A00E9F09000031214309002B2F0122E73804B
:10127A006E121A217B017A027964900274EBF0A350
:10128A00EAF0A3E9F09000031214309002B2F012CF
:10129A002A95122D551229F68045121A217B017AB8
:1012AA0002796490027AEBF0A3EAF0A3E9F09000E5
:1012BA0003121430FF900004121430FD900005123E
:1012CA001430FBC00390027AE0FBA3E0FAA3E0F932
:1012DA00900006121430900293F0D00312193512BE
:1012EA002E0A02110C121A217B017A0279649002E9
:1012FA007AEBF0A3EAF0A3E9F0900003121430FFAE
:10130A00900004121430FD900005121430FB1217DD
:07131A0075122E0A02110CEE
:102CA30075FFDE75FFAD75B207122B17122C2E12AE
:0B2CB3002DAE122E5A122E20021A091C
:0A2E2000759A07759D0475F80322EA
:102B1700E58954F04401F589D2A9D28C438E60D25D
:102B2700ADD2BD43E70443F70475CA1175CBFE75F3
:062B3700E41375E5FE2227
:102C2E00E4F5A775B0FF75BDFCF5A57590FF75A40D
:0E2C3E000D7580FF75A6FF75E10375E340225A
:102DAE0075AB1975AA8075BC3875E8C175D10B2243
:072E5A0075D49C75D794228A
:102D840075AC38EF2438F5AC75AA8075AA90E5AA1D
:052D940030E5FBAF9CDF
:012D99002217
:0D2DCD008FBB75E8D1E5E830E5FBAFBF2214
:1029F600AF4F90033A7480F0E55530E204EF44108F
:102A0600FFE55530E104EF4420FFE55530E004EFE3
:102A16004440FF301E04EF4480FFE55520E304EFF9
:052A26004401FF8F9B3D
:012A2B002288
:091A090043E60875D983D2DE2200
:031A1E0002226B36
:10226B00C0E0C0F0C083C082C0D075D000C000C039
:10227B0001C002C003C004C005C006C00720DF03B5
:10228B00022339E50945086008E5091509700215AF
:10229B0008E54445436011E54415447002154314A9
:1022AB0045437004F54FD220E5B05407F526654E33
:1022BB00600CE526654EF532753C0385264EE53CF4
:1022CB006035153CE53C702FE53230E010E52620FB
:1022DB00E00B900313E4F0A3744BF0D21FE5323004
:1022EB00E208E52620E203752704E53230E108E534
:1022FB002620E103752702301F32900314E024FFE0
:10230B00F0900313E034FFF0E5B030E005752701E2
:10231B00C21F900313E07002A3E07010C21F900362
:10232B0016E0FF7BFF7A2E7934122873C2DFD007B9
:10233B00D006D005D004D003D002D001D000D0D02D
:09234B00D082D083D0F0D0E03242
:0C2DE700754F04D220754300754464222F
:0C2DF300754F02D2207543007544642225
:102C5400420262000042020D00004202080000C16C
:052C640024C123C12280
:0A2E2A00C223C224E490020CF0223F
:102B8800E4900262F0A3F090020DF0A3F0A3F0909D
:102B98000208F0A3F0900203F0A37440F0E490025E
:032BA8000BF0220D
:062E6100122E2A022B884C
:102D0C00E4F5848FC343C30175C04475CF8EC2C331
:092D1C0043E60290020A04F022D1
:101A2100E4F58420C7FDC2C2122E61E490020AF0DF
:011A31002292
:0B2E0A00E4F584D2C290020A04F0221A
:0D2DDA00AE07122D0C900207EFF0022E61E3
:102B6300E4900337F0A3F0302302FF222024FDD2A8
:102B730023900205E4F0A37410F0900250EFF0E408
:042B8300A3F07F013B
:012B8700222B
:102A610030230A900205E07002A3E070037F002288
:102A7100900206E024FFF0900205E034FFF090029E
:102A810051E0FE04F074522EF582E43402F583EF36
:042A9100F07F0122AF
:0B2E1500302307C223D224122DBE225E
:0E2DBE00AF84E4F58420C7FDC2C4D2C58F8463
:012DCC0022E4
:102723009002F4EBF0A3EAF0A3E9F090020AE07060
:1027330002FF229002F7E0FE6005D3941040037F6E
:082743000022122B63EF604E2F
:10274B00E49002F9F09002F7E0FF9002F9E0FEC38B
:10275B009F50249002F4E0FBA3E0FAA3E0F98E82F1
:10276B00758300121430FF122A61EF7002FF229062
:10277B0002F9E004F080CEE490020CF0122E1590DA
:0E278B0002F8E070032024FD90020CE0FF2213
:032799007FFF229D
:0E1E6800900317EBF0A3EAF0A3E9F0A3EDF06E
:101E7600E4FFD3900263E09400900262E0648094F1
:101E86008050012253E6FD900208E0FEA3E0240FF5
:101E9600F58274023EF583E0FF900208E475F001D6
:101EA6001214D9FCE5F064404C7006900208F0A3C9
:101EB600F0900204E004F07006900203E004F0E4FF
:101EC600FE90031AE0FDEEC39D5054EEC39F504FA3
:101ED600900208E0FCA3E0240FF58274023CF5832F
:101EE600E0FD900317E0FBA3E0FAA3E0F98E82750C
:101EF6008300ED12146F900208E475F0011214D9F4
:101F0600FCE5F064404C7006900208F0A3F09002E5
:101F160004E004F07006900203E004F00E80A2EEE6
:101F2600C39F5029900208E475F0011214D9FCE50C
:101F3600F064404C7006900208F0A3F0900204E0B2
:101F460004F07006900203E004F00E80D290026363
:101F5600E024FFF0900262E034FFF043E6029003D3
:0C1F66001AE0FEEFC39E50028002AF069E
:011F7200224C
:102D2500D3900263E09400900262E0648094804056
:082D3500047F0180027F0022EF
:031A1800021D0AA2
:101D0A00C0E0C0F0C083C082C0D075D000C000C09F
:031D1A0006C007F9
:101D1D00C225AFC1EF1215051D53081D53101D63CC
:101D2D00181D68201D75281DA2301DAD381DB5600C
:101D3D001DB0681DB5701DB0781DBD801DBD901EF8
:101D4D0034A000001E42900250E0F5C2C2C59002C0
:101D5D004FE4F0021E44900251802890020C74FD55
:101D6D00F0D2C4D2C5021E44900251E0FF90024F42
:101D7D00E0C39F5014E0FF04F074522FF582E43459
:101D8D0002F583E0F5C2021E44D2C490020CE4F0C9
:101D9D00C224021E44D2C590020C74FEF0021E44F1
:101DAD00021E39D222021E44900202E4F0021E44A9
:101DBD00900202E07020E5C2F0E0FFC3900204E063
:101DCD009F7480F8900203E06480985003122B8872
:101DDD00900202E004F0900204E024FFF090020370
:101DED00E034FFF090020DE0FEA3E0240FF58274C5
:101DFD00023EF583E5C2F090020DE475F001121478
:101E0D00D9FEE5F064404E700690020DF0A3F090FF
:101E1D000202E014F07020900263E004F07018905C
:101E2D000262E004F0801030220DC22290024FE4D5
:101E3D00F0D2C58002D22530250EC2C6D2C6C2C58B
:0A1E4D00C2C4D2C2C225C224C2C31F
:101E5700D007D006D000D0D0D082D083D0F0D0E049
:011E67003248
:052E6700A2C7E433FFE7
:012E6C002243
:0E29B100900307EBF0A3EAF0A3E9F0A3EDF02A
:1029BF00E490030CF0900307E0FBA3E0FAA3E0F927
:1029CF00A3E09002F7F090030BE09002F8F0E4FF21
:1029DF00122723EFB4FF0D90030CE0FE04F0EEC3BB
:0629EF00940340D17E00BC
:0129F50022BF
:0B2AC40090032BEBF0A3EAF0A3E9F075
:102ACF007E007F007D1012152B90032BE0FBA3E0FF
:102ADF00FAA3E0F97D10121E68EF7002FF227F014A
:012AEF0022C4
:102873009002BD7422F0A3EFF0A37413F0121417A7
:102883009002C0F09000011214309002C1F0900049
:10289300021214309002C2F090000312143090021E
:1028A300C3F09000041214309002C4F0900005129B
:1028B30014309002C5F09000061214309002C6F056
:1028C3007B017A0279BDE490030BF07D0A0229B102
:102BCD0090031B7422F0A3EFF0A37403F0A374FF22
:102BDD00F07B017A03791BE490030BF07D0402294D
:012BED00B136
:102BEE0090031F7422F0A3EFF0A3741CF0A374FFE4
:102BFE00F07B017A03791FE490030BF07D04022928
:012C0E00B114
:102C0F00E4900323F0A3EFF0A3740AF0A3EFF07B9B
:0F2C1F00017A037923E490030BF07D040229B1BD
:062E6D00C2C253E6FD2283
:101A36009002D1E0FFA3E0FCA3E0FDA3E0FBA3E05E
:101A4600FAA3E0F990028AE55FF0E560A3F0900260
:061A5600D9E090028CF0C3
:101A5C00900284EFF0A3ECF0A3EDF0A3EBF0A3EA7B
:041A6C00F0A3E9F00A
:101A700090028D7403F0A374E8F0A3E584F0E4F51C
:101A80008420C7FDC2C4D2C2D2C5E4FF90033CF09B
:101A900030C3FDAEC1EE24F8602324F8601F24F8A3
:101AA000602F24F8603624F8603A24F87003021B93
:101AB0004824F87003021B502438021B58EF700CA6
:101AC000900284E025E044A0F5C27F03C2C5021B5A
:101AD0005E900285E0F5C27F05021B5E90033C74B8
:101AE00003F0807AEFB4050B900285A3E0F5C27F86
:101AF00006806BEF6406703E90028CE09002877067
:101B00000FE0FBA3E475F0011214EFA9F0FA8008CE
:101B1000E0FBA3E0FAA3E0F9121417F5C290028BE0
:101B2000E024FFF090028AE034FFF0E07002A3E0CE
:101B3000702C7F078028EFB40706D2C47F09801E6F
:101B400090033C7405F0801690033C7404F0800E02
:101B500090033C7406F0800690033C7401F0EFB4EF
:101B60000904C2C3803690033CE0B4031C90028D8C
:101B700074FFF5F01214D945F0600ED2C4D2C5D26C
:101B8000C2C2C3E490033CF0FF90033CE06008C293
:101B9000C5D2C4C2C38005C2C3021A9020C7FD903B
:051BA000028FE0F58456
:011BA500221D
:101BA60090029CEFF0A3ECF0A3EDF0A3EBF0A3EA18
:041BB600F0A3E9F0BF
:101BBA009002A47403F0A374E8F0A3E584F0E4F5BA
:101BCA008420C7FDD2C2C2C4D2C5E4FF90033CF050
:101BDA0030C3FDAEC1EE1215051C08001C0B081C13
:101BEA000B101C36181C41201C49281C64301C6C24
:101BFA00381C74401C84501CB65800001C08021C77
:101C0A00BCC2C5EF700F90029CE025E044A0F5C26B
:101C1A007F03021CC2EF64016003021CC290029C93
:101C2A00E025E044A1F5C27F04021CC290029DE0B7
:101C3A00F5C27F05021CC290033C7403F08079EF61
:101C4A00B4050B90029DA3E0F5C27F06806AEFB44B
:101C5A000606D2C57F018060801890033C7404F0A8
:101C6A00805690033C7406F0804EEFB404047F0261
:101C7A00804690033C7405F0803E90029FE0FBA3EF
:101C8A00E475F0011214EFA9F0FAE5C212145D909E
:101C9A0002A3E024FFF09002A2E034FFF0E0700219
:101CAA00A3E07004C2C280107F02800CD2C47F09F4
:101CBA00800690033C7401F0EFB40904C2C3803675
:101CCA0090033CE0B4031C9002A474FFF5F01214D4
:101CDA00D945F0600ED2C4D2C5D2C2C2C3E49003C1
:101CEA003CF0FF90033CE06008C2C5D2C4C2C38086
:0F1CFA0005C2C3021BDA20C7FD9002A6E0F584E5
:011D090022B7
:10207B009002D1EFF09002D4EBF0A3EAF0A3E9F0D9
:08208B009002D2ECF0A3EDF08D
:10209300756100543FF562543F605CC374409562C0
:1020A300FFE49561FE9002D7E0FCA3E0FDC39FEC43
:1020B3009E50068C5F8D6080048E5F8F60121A368F
:1020C30090033CE060037F02229002D3E02560F09E
:1020D3009002D2E0355FF09002D9E0700B9002D508
:1020E300E55F8560F01214D9C39002D8E09560F0E3
:1020F3009002D7E0955FF09002D7E0F55FA3E0F59B
:1021030060D3E5609400E55F94004070E56094401F
:10211300E55F94005013121A3690033CE060037F8E
:102123000222E4F55FF56080D89002D1E0FFA3E0DE
:10213300FCA3E0FDA3E0FBA3E0FAA3E0F990028A8D
:10214300E4F07440121A5290033CE060037F0222D1
:1021530074C02560F56074FF355FF55F9002D3E0CE
:102163002440F09002D2E03400F09002D9E0709164
:0E2173009002D575F0401214D90221047F00AD
:01218100223B
:102D6D009002A2E4F0A304F0121BA690033CE060D5
:072D7D00037F01227F002209
:102CBE0090033BEBF07B017A03793B9002D7E4F073
:0A2CCE00A304F0E4A3F012207B221F
:102BAB00C0079002E9E0FFA3E09002A2CFF0A3EFF1
:102BBB00F0D007121BA690033CE060037F01227F3D
:022BCB000022E6
:102CD800C0079002F1E0FFA3E09002D7CFF0A3EF86
:0A2CE800F0E4A3F0D00712207B22D5
:082E3C00002400300018000C16
:031A12000228089F
:10280800C0E0C0F0C083C082C0D075D000C000C096
:1028180001C002C003C004C005C006C007C082C012
:1028280083852A82852983740193F5D2E493F5D3AD
:10283800A3A353830F43838085822A858329D0836A
:10284800D0823017098540CAE53FF5CBC217C2CF01
:10285800D007D006D005D004D003D002D001D000D4
:0B286800D0D0D082D083D0F0D0E0327E
:031A330002279CEB
:10279C00C0E0C0F0C083C082C0D075D000C000C003
:1027AC0001C002C003C004C005C006C007C082C07F
:1027BC0083852D82852C83740193F5D5E493F5D60E
:1027CC00A3A353830F43838085822D85832CD083D1
:1027DC00D0823018098542E4E541F5E5C21853C9A9
:1027EC007FD007D006D005D004D003D002D001D0C2
:0C27FC0000D0D0D082D083D0F0D0E032EA
:031A0600021F7349
:101F7300C0E0C0F0C083C082C0D075D000C000C034
:101F830001C002C003C004C005C006C007E5553048
:101F9300E303022060758CF2758AFB301B0EE53E6D
:101FA300253BF53BE53D353AF53A800DC3E53B95D9
:101FB3003EF53BE53A953DF53AE55530E1113021E3
:101FC30004C221800A5008753A00753B00D22153A0
:101FD30033C3E53AC41313540325E0FFE433FE741B
:101FE3003C2FF582742E3EF58374019342331228FD
:101FF300D3E55530E010E53A90033DF0F551F4F5A3
:10200300525333FC8034E5536006D553035333FEF8
:10201300E5546006D554035333FD301A1DC21AB27A
:102023001930190C433301755305E530F551800A16
:10203300433302755405E530F55290033DE4F0D384
:10204300E53E9403E53D64809480400E301B0574A7
:1020530004F0800690033D7402F08533A0D007D0CE
:1020630006D005D004D003D002D001D000D0D0D008
:0820730082D083D0F0D0E032EE
:1028D300C3E53B9531FFE53A9530FED3EF954DEED9
:1028E300954C4037301B0EE54D2531F531E54C3520
:1028F30030F530800DC3E531954DF531E530954C1C
:10290300F530E55530E110301304C2138009500748
:0C291300E4F530F531D213D21A80B52261
:108000008953AA7A83C6D9FAD4BBEB0EA37DD44A8E
:10801000B740CC0093CCD59CBBACBF9E6A3A93577B
:10802000756A8FCB6286B2AAA822BA346FA19ED994
:1080300081C39813630CA99695D1A131544786A5A5
:10804000727596BC7334CC95CA7DE3E69F52D2FB21
:10805000B8A2CFE299F6DDCFC5A5CB1276DEA0D9C6
:1080600083789E1270B1C065B51CC61C7A2BA7BD63
:1080700088BD9CE66580A97C93009B894BB07B11F1
:1080800063DE85275EAEB535B062C73A8047B1CAB8
:10809000958EAB3473FEB6E39E1FA3524F4579CE47
:1080A0005D6179554DB69F9196D1AABB620F933C05
:1080B000782790845D94A63F94A3A233577F8C17B2
:1080C0007A24A0AA7F62DB02DB27F6C9B46AEA42FF
:1080D000D211EB70B79AFD7EE752EEB09C5EC82BD2
:1080E000AC8DC8D59D11EE4EE478F6D6AC2CDAED09
:1080F000BD04D22B9BA8E06ECAA0D3BC845BB4168F
:108100009D22BE8C9816EE84E97BFFFFB89AE99019
:10811000CCA8E187A96CEB51D171D56D800FA92C4A
:108120008B3AA591783DC84CBDABCF9D84E6B3F4A6
:1081300096AFACCA7789BDD4A9CAB4E067A799B095
:108140008526A90D8520DE18DB90F485AF77E2A1A6
:10815000C7C4DE7CA802EB49D287D7588283ABD84C
:108160008DCDA7B879A4C8A1BC9CCCDD8028ACF18A
:108170008D26A07F6846AB6B94159BC04B07798416
:10818000616A81C95A63AFFBAA37C01B7831A8BDA9
:108190008B86A03067FCA9E2901D944E3F3F68C3D8
:1081A0004B516640399B8A7080A9938D49DA7A00D9
:1081B0005DE5753D414888F0765182DF372A6AC314
:1081C00057D37D5E5B1BB5C4B4F3CFA38C53C13EC4
:1081D000A821C0998BDDD0E0B9D5C0596D2F982A60
:1081E0007BBB97396AAEBB28B094C23876D9A4E974
:1081F00086559AD563B2A7DC91789A034A16794CD2
:1082000061D782C75BDEB1DEAC6DC28F7ACFAB7057
:108210008E3AA2D06A74AC1D920995D84053695029
:108220004B45658A382B88367D978F9344ED7412C1
:1082300056EC6D2D38197E976AC9762129315B8AF3
:1082400047566B9C4814A1779F62B8D17443A7F43A
:108250008DA5A4F16F12B2FA9AE0A0604C3E764F61
:10826000590573B6466F963F8B129C30505F7E1255
:108270005F3573823C4180646A1172C4231752A433
:108280003BA05D1836CF8D8988EA9FF7593A8AF569
:108290006EF184D24DD790F878727DE52A1954E2B8
:1082A00038B854F029977BB8734087723F107087B5
:1082B00055BE6E683BC684C07374815536F36BDD62
:1082C0005A3E811A6026BC1EBC99D895968ECCC0A9
:1082D000B4EACEA59B2BE16CCB9ED35B8168AD95B8
:1082E0009257AF01839FD53FCBCCDE8D9448C36DB1
:1082F000A5EABB76855ACA86B520BEA46FAB9FCED1
:108300008943AB16850ADBE2D743EE32A738D8980B
:10831000BC1CD16699B7DC07C293C6FB72099B935C
:108320007E0D98D16BE9BC65B22FC48F7A44A9BE8B
:108330008CE5A36C6E97B54EA1B0AD32606492D857
:108340007EB9A30B7F88D8EAD6CCF02BAB86DF1999
:10835000C4A5DBC4A5B2E960D105D63D81CDAB880B
:108360008DE2A8317A81C9E2BE3FCEE2828EAFB9FA
:0D837000904EA4066C2CAFAF98B7A0BF5084
:10837D00627F3A677B88346127B717B1AAC7E5805A
:10838D0051B131944EA94C716AB3A09A2C9EAC494F
:10839D00EB73BD569871D2457796958D17A04256C1
:1083AD00D687416B6A83054F52973A84DB91A84675
:1083BD00317A0667518D166B0CC5EDC552E0379DB0
:1083CD001CD239B94ED1F69D6AE29ACBBCD26B7FE5
:1083DD006BAA8F8E48A9EC7D86CE23C3B1D5778A43
:1083ED0037B86699EFAE8B7782BBC5A579AE1A5EAD
:1083FD00438D8C762A972B7051C660C0FCD72A8F7F
:10840D0074C01EA2EFB78C7F35C0E2A6D0AA9F55CF
:10841D001A7E1560077A474CE29CE6923EA43159CC
:10842D007F88986B6381954C7092DD7EFB8A3F3D12
:10843D00396F7A5B2F7F5B5BB7B4FEB2CCCC1B87F9
:10844D006DBAFDA08BB7B381AFC571AD2FB2855E8F
:10845D003A881F6AA9852C57B7A7569BF8ACE460DC
:10846D00E08E5E6F4B83614BE98FD3794581BD31D2
:10847D00D4612449E16B1A44919B099628ACF165AE
:10848D00F097667B1C90B659739C4B837B88A33405
:10849D008C5F0942925E7C32D384A57BDD8FBE4713
:1084AD000A782E5D12756842718B16797486FE3CC2
:1084BD004470D75EE085626415BFB2BFD3DB73999C
:1084CD0011CEE7B6B4D0129C3AE21DCBF1D34F805A
:1084DD00FDACCB912DAD7781B5D2F4C920DB819068
:1084ED00DABF9EA1B9B6E38066C52FAF67B88869BC
:1084FD002D98EE8200A3717D02D378CE76E5039D93
:10850D00A6CEA4B1C6C6AE8E9DD08BB6B6BABD658D
:10851D006A8E9270AC8B0F5DC7ADE3A34EB54E6AFC
:10852D00A499C07C8992B35D80A3DA8FE09B064D40
:10853D00DD7FF66B7C8F756B99C4A2C22CDB3396F5
:10854D0038C975AEABC5768F0FD26AB9BCBEA269FC
:10855D00E1934C75568F566158B06BA47CB4D468BA
:10856D00369516756288D350B293EF7CB28476330C
:10857D00D6626C4A6C6AE54399994B93A2A9A061A6
:10858D00D29278755D8A23520B940D7A657EB3294C
:10859D00C05362360D511A249275856BDD7EDF3521
:1085AD004B65904995610C2D3774FE627F6F2D23BD
:1085BD0099575344836A2F480EA2D8A229BCFB7940
:1085CD00CDAED995E0AE7A79E1BF06A81FAEC65BF8
:1085DD00C086DE6A93863559CEAA6C9FFCB1C566FE
:1085ED008B94C076518AF653F9984882098ABA3A23
:1085FD00F46A4F530174174D54A37B9E31B47A6CBA
:10860D00E19DA9809A95575D239EF4850788FE33D9
:10861D00A15CC63EE459502C1A7C4D71D683FB39B2
:10862D007E68CC4BCE62392D4D73F560506BD11FEA
:10863D000A518C3D8361F23E9398219635AFCD6BF7
:10864D006A9F4585209C9566E1AAF3930398AC44F7
:10865D00B56EF051D06CAC3F8F8F89848695D04A22
:10866D0029780659536DCB36B57B0264D96DB71E8B
:10867D00344DEC371258B53296897A85069C3D55A6
:10868D00AA87906BB781C14AF18E3D75E17B7E273C
:10869D00DC52D036D0533228027A4E71FF865C3EC2
:1086AD00236FC455256DF83B8084A47381818B376E
:1086BD00526C665AF181F5612BBD4BBDF0DA139802
:1086CD0036CE91B6E3D0C69D75E3DECE37D61D848A
:1086DD0052B0A79590B2628728D8EFCFA3E28C98BD
:0D86ED006DC7B9AA5DC0108A1BCF6DBA2DF4
:1086FA00C3D77504A54D8EE7B0E08AFAE1F7DD7DB0
:10870A00F491ADBCDF41C2E9D857A0CCE341C9F12D
:10871A00CE7D79AEA35B85F9A0DF741AC4B9BAA677
:10872A00CD2782FEB29A95E3AC8D77D9BEB1AB3331
:10873A00B6D66A299CBD88BEAD3189CEE34FE150D9
:10874A00FACEB648E9FACFA4E6E2B0EEF4BADC7C97
:10875A00E1D28D7FB75799CEB43986A6D622CA9B65
:10876A00DB598F22BC679D17B0EA792ABCC7A5E9F5
:10877A00AE0B5DC78CB8751295E36EEFC4F7BFA256
:10878A00D5F48E77BF6FA2A3B7B67FEBC237A8D94D
:10879A00AD6F58C282A9659880E754A0A5D29C689B
:1087AA00AFA5664C96CA7B0692B25F12A70B94BD20
:1087BA00A19B56348A1A77759D497B4FD63FD5B30C
:1087CA00F0A7AD99E2C4C9E7E29CAE1DF35ADC8872
:1087DA00E3439050BB7F9F43BAF28E96DF3ED4D6D6
:1087EA00E6A59B6FC9A7AB38BFDD88DCCD26B6E10D
:1087FA00BF8A6FB99F0987ADA8B481DFD7F3D29436
:10880A00E8C6A115D1C2B497C93790E2D292B8820C
:10881A00BC5366D08FCC71BF8BFF5E9BAE9EA3F616
:10882A00B5E86B349A4C7D1693455E1EA48890A3D6
:10883A009BE34ED981166CC690ED6D45C686C44E33
:10884A00DD9798E3CC6BB1F2C9129307D6C0BE7517
:10885A00C3C36F6F994A7BC9964368C3B857ACEED6
:10886A00BDCE71BE9F2F801094195C93A06F89D4DE
:10887A00923D424571865A347B5E54C4AB2CA63A6B
:10888A00BCF375E0A7448AE8A06F691AABDF92FCD3
:10889A00981043E46E4D51C16D9641D893948AB6AF
:1088AA009E8155B686C36B9083CE50BF994B8790F5
:1088BA0095024A2F7EA86C9692FE7197CD19CD1F0C
:1088CA00E8A3A625DBDFC38FDCD0A8DCEEA1D8574E
:1088DA00DF978D27B8D69D19B9448D62DE81D48D74
:1088EA00E6CD9C05CAA8ACA1C1AA8B0ACFB2B9C76A
:1088FA00C2C57346A2E48BD2AD1E868BDCDCD7B62A
:10890A00EE1DA69BD773BA6ECF3096F8D8C0BEC3F9
:10891A00C2A26D2796277819925364E2B4D5AA1792
:10892A00BBED7119A00A82A998A8634AA97995533F
:10893A00A04D52F884E5703E940A7001C8DDC63A2B
:10894A00DF1399E9CCF8B1FFC89B9206D531BC5424
:10895A00C10A6C199553772D90FD62CEB1B0A590DE
:10896A00B5B668E6959575AF88ED509993A47C33B2
:10897A0083C432F16153491F696441E49762918467
:10898A00A74E5F4A8FBC726B86FC4EAE907A769C7D
:10899A007AB3258A4EF5316A4C401F82703D665E75
:1089AA0079282F5D5F6A43365A7526686DF75B3FF3
:1089BA0067B51BE84F693C6061D33F789A099920F3
:1089CA00B3B87050A5238BEFA44F6F7CB4669D4457
:1089DA00A3B150707B535ECE7A344D929DF5934A83
:1089EA00A4D75961875B68B07D1A45E089F373792A
:1089FA007BEE2BEB5B0B4380645A3D5B93458DBE4C
:108A0A00A3CB5BF58C806F3583B64B448CD972AFA0
:108A1A00766920CF49B72B9845C81854684A5D969D
:108A2A006F7E24C353D5369A4CC7179F5E0A4A27CE
:108A3A00556B08673AAD26664A9826FC804D7E2417
:108A4A00977F52DF867D6C1B83544D629137790A7A
:108A5A007E772A44544236E55185242C73E968AA64
:0D8A6A0079B72DD45B753C8650C119705D45
:108A770081471C4FBE00002F7C186739CE13756ADB
:108A87001E656E7C6A359D67474B34610429F96D15
:108A97000A547459D705FB30B5147C30A4053B57ED
:108AA7004D4EC662E91A774BDF310849A316F25FCC
:108AB700DE4E835C5611E546C135145BE13AE0961C
:108AC700C99737B3257111A7358F51A8FF7578BBA3
:108AD700ABA5D0AD805B8087A16C5688F35D85AF71
:108AE70018A599B84E6DFC9D167F8695075EDFA386
:108AF700FF8E8D9806490179196283844B5E34B5E0
:108B070001B057C73B8036B18C9505AA44728BB428
:108B1700D19B539FB14AB6743556A6715F446E9484
:108B2700E18AA29CF852A4821565337BB246D38DA5
:108B37008279DB8554387E6AEA56C27B0D5782B04C
:108B4700DCAEB6C80C8360B6EC9C70B3887D6FC191
:108B570016A8B3ADE4596E832265767FBE5208A18D
:108B67006195B9A65559FC872067AF7B6243828719
:108B7700007002780527A256753EB15F6538538E9F
:108B87003E88CD9F03576A88466B5F805848728A34
:108B9700A5712C75A920E44AB22D8948C01C626DC5
:108BA7007D63FC77232DB45E1C424359DB26266E7A
:108BB7000C5BAA68751CFC50CF3E1863DB41CF9C49
:108BC700AE9C12B6F673D9A8F49009A8AF7422B96F
:108BD70051A273A9215621814464FD80A0543AA46F
:108BE700D89A66AC2C60ED8F1C70A585424E3A92E0
:108BF7007D7C3184D434FE64484CE76DEA47119D8F
:108C07002197BFADEF663B96E679BA8E5956049722
:108C1700B37DA481762BF354F136E6512923C7732C
:108C2700CD69297B1F30705F8D425C589223706934
:108C3700E15603614B1449468F3248567932DA8C34
:108C47002689F8A34C5EA3923877CB8EF958FA9C05
:108C5700C1848589E1359C5F8642165CA02F307EF2
:108C6700D6737E8471387365F846EC5B0923976782
:108C77008851025981099F38F721BB42FC1C7B723E
:108C8700FB6E2184F33DF96F78533668D8319E74B3
:108C97007F5BB860E80CDA37601AF236E50B465DA1
:108CA700215462684D1FA250D035BE4E1E1B316342
:108CB700E052485FDD152D49CB37DE5E6B3D2998C5
:108CC700D098FDB4A87251A832900AA97475A8BBB0
:108CD70096A575ACE05A9986746AE287385B82ACD0
:108CE700CDA306B5736AD999AA7BD191095A989FE2
:108CF7006F89B492E3439473635C837E0157A0AE9C
:108D070023A930BFCA787CA9888CB8A1AE69ACAB5F
:108D1700A991E295F840B369EA4C146685394D8903
:108D2700787EF3910246687593586C6EA539837FF8
:108D3700ED6C0277382A1F5C4947DF6BE9481DA1B4
:108D4700379ED2B7E972FFA64D8B94A2706C1BAF0A
:108D57008796EA9BE1473270AE52CB6CDD3EF18ECF
:108D670016823992A246167309536866EB2EDD7296
:108D77002D5B0262D9124B40F429084994225B7893
:108D870020728A889C40E1719B5494696E316A73A2
:108D97007F59EB5E4D096E332415E4310504925576
:108DA7009A4C065F1D159E45F72A11419D0DDD550D
:108DB700B9434F50130495386325AA4B6B295F8439
:108DC7004083A69E8E5B76909877B590655BE2A10F
:108DD7001E8A4D910A3E1B694F4D1C68D43C848DF9
:0D8DE7003982E094C0499D77E959926E4EA3
:108DF40037687BCE65A76E701EC14E3436FE582C84
:108E0400318187C0828D98EF516E824E65577A2DDD
:108E1400421183FB6A276E3618F2423024663EEC18
:108E240011CE621B57BD69FB1F974EFE321A489E36
:108E340013CC5A8D4701529C05EF388B249C49254D
:108E440025E07F877DB69768531F87146D09849941
:108E54004EFF932C7B56811A2D3E57933A8E55859F
:108E6400288378986DB07F143389618142EA577CF6
:108E7400208264EA4EDD57D6086F3842218443428B
:108E84001D4074406FE7873A40C372C557086D2F81
:108E9400367A79E261A3675B13D63EE623033F810A
:108EA400146E66D65EA5731E2B025CBF423D5B2E1C
:108EB40028D27213610D6F3425195A4A48F1701281
:108EC4004F66ABA3AC65C8A686E6BD5EA5CEBFCF94
:108ED4008C9BD322BD99C59C73EFA0628569A2596E
:108EE400773CC921BFF3D2FA88FAB8649B26B0F75D
:108EF4007B20C090AB6FB537668296EA80A3A2BA96
:108F04007CF2D40ECFB2E6E4A02ED1D2B599CB2612
:108F140093BAD64DBD1BC1C66D1796E2799F94A432
:108F240067FFB8BCAEC8C169775FA71A8A82A14B34
:108F34006CB6B3ADA04FAC115F8392377E57A2E9F4
:108F44007FA5D946D767F104AC9EE06FC639DD979B
:108F5400A7C2EBAED390D90584D2AECA9160ABEB75
:108F64007E78CE14C2ADD38B8773B4D895A8A99B51
:108F740071FBB5B89EF9A73B571886296EA38F9449
:108F840068BFBEE8B9B3D02588C9B9E09D34B268DA
:108F94007ABCBD29A3EBA8A154157E1C612B7C9A35
:108FA4005074A1C6987CABDA62A1933F779B8F681B
:108FB4005BE7A40191D49ED2538C8792750D9B02DA
:108FC4007928D438D3CDEEE1ABF4E13FC882E1583F
:108FD400ACF9F256DBA5E2818FAEBAFD9EE2BAB1DE
:108FE4008E76DF3ED4F6E6E69BD0CA28ABDAC09F85
:108FF40089BFCE2AB805C0CE711EA08EFC1CFC1FF2
:10900400FC23FC26FC2AFC2DFC31FC34FC38FC3B04
:10901400FC3FFC42FC46FC49FC4DFC50FC53FC5715
:10902400FC5AFC5EFC61FC64FC68FC6BFC6EFC722C
:10903400FC75FC78FC7BFC7FFC82FC85FC88FC8B4B
:10904400FC8FFC92FC95FC98FC9BFC9EFCA2FCA56E
:10905400FCA8FCABFCAEFCB1FCB4FCB7FCBAFCBD98
:10906400FCC0FCC3FCC6FCC9FCCCFCCFFCD2FCD5C8
:10907400FCD8FCDBFCDEFCE0FCE3FCE6FCE9FCECFD
:10908400FCEFFCF2FCF4FCF7FCFAFCFDFD00FD0235
:10909400FD05FD08FD0BFD0DFD10FD13FD15FD186F
:1090A400FD1BFD1EFD20FD23FD25FD28FD2BFD2DB3
:1090B400FD30FD33FD35FD38FD3AFD3DFD3FFD42FC
:1090C400FD44FD47FD49FD4CFD4EFD51FD53FD564C
:1090D400FD58FD5BFD5DFD60FD62FD65FD67FD699D
:1090E400FD6CFD6EFD70FD73FD75FD78FD7AFD7CF4
:1090F400FD7FFD81FD83FD85FD88FD8AFD8CFD8F4F
:10910400FD91FD93FD95FD97FD9AFD9CFD9EFDA0AF
:10911400FDA3FDA5FDA7FDA9FDABFDADFDAFFDB212
:10912400FDB4FDB6FDB8FDBAFDBCFDBEFDC0FDC27B
:10913400FDC4FDC7FDC9FDCBFDCDFDCFFDD1FDD3E4
:10914400FDD5FDD7FDD9FDDBFDDDFDDFFDE1FDE353
:10915400FDE5FDE7FDE8FDEAFDECFDEEFDF0FDF2C9
:0D916400FDF4FDF6FDF8FDFAFDFBFDFDFD3F
:10917100FFFE01FE03FE05FE07FE08FE0AFE0CFED1
:109181000EFE10FE11FE13FE15FE17FE18FE1AFE4E
:109191001CFE1EFE1FFE21FE23FE25FE26FE28FECE
:1091A1002AFE2BFE2DFE2FFE30FE32FE34FE35FE52
:1091B10037FE39FE3AFE3CFE3EFE3FFE41FE43FED7
:1091C10044FE46FE47FE49FE4AFE4CFE4EFE4FFE61
:1091D10051FE52FE54FE55FE57FE58FE5AFE5CFEED
:1091E1005DFE5FFE60FE62FE63FE65FE66FE67FE7B
:1091F10069FE6AFE6CFE6DFE6FFE70FE72FE73FC10
:1092010088FC8BFC8DFC8FFC92FC94FC97FC99FCF8
:109211009BFC9EFCA0FCA2FCA5FCA7FCA9FCACFC51
:10922100AEFCB0FCB2FCB5FCB7FCB9FCBCFCBEFCAE
:10923100C0FCC2FCC5FCC7FCC9FCCBFCCDFCD0FC0E
:10924100D2FCD4FCD6FCD8FCDBFCDDFCDFFCE1FC71
:10925100E3FCE5FCE8FCEAFCECFCEEFCF0FCF2FCD7
:10926100F4FCF7FCF9FCFBFCFDFCFFFD01FD03FD3B
:1092710005FD07FD09FD0BFD0DFD0FFD11FD13FDA5
:1092810015FD17FD19FD1CFD1EFD20FD21FD23FD12
:1092910025FD27FD29FD2BFD2DFD2FFD31FD33FD85
:1092A10035FD37FD39FD3BFD3DFD3FFD41FD43FDF5
:1092B10044FD46FD48FD4AFD4CFD4EFD50FD52FD6D
:1092C10053FD55FD57FD59FD5BFD5DFD5EFD60FDE7
:1092D10062FD64FD66FD68FD69FD6BFD6DFD6FFD61
:1092E10070FD72FD74FD76FD78FD79FD7BFD7DFDE0
:1092F1007EFD80FD82FD84FD85FD87FD89FD8BFD61
:109301008CFD8EFD90FD91FD93FD95FD96FD98FDE3
:109311009AFD9BFD9DFD9FFDA0FDA2FDA4FDA5FD68
:10932100A7FDA8FDAAFDACFDADFDAFFDB1FDB2FDF0
:10933100B4FDB5FDB7FDB8FDBAFDBCFDBDFDBFFD7A
:10934100C0FDC2FDC3FDC5FDC7FDC8FDCAFDCBFD06
:10935100CDFDCEFDD0FDD1FDD3FDD4FDD6FDD7FD94
:10936100D9FDDAFDDCFDDDFDDFFDE0FDE2FDE3FD24
:10937100E5FDE6FDE7FDE9FDEAFDECFDEDFDEFFDB7
:10938100F0FDF2FDF3FDF4FDF6FDF7FDF9FDFAFD4B
:10939100FBFDFDFDFEFE00FE01FE02FE04FE05FEDC
:1093A10007FE08FE09FE0BFE0CFE0DFE0FFE10FE71
:1093B10011FE13FE14FE15FE17FE18FE19FE1BFE0C
:1093C1001CFE1DFE1FFE20FE21FE22FE24FE25FEA8
:1093D10026FE28FE29FE2AFE2BFE2DFE2EFE2FFE46
:1093E10030FE32FE33FE34FE35FE37FE38FE39FEE6
:1093F1003AFE3CFE3DFE3EFE3FFE40FE42FE43FE87
:10940100B1FEB4FEB7FEB9FEBCFEBFFEC1FEC4FE96
:10941100C6FEC9FECCFECEFED1FED4FED6FED9FEDE
:10942100DBFEDEFEE1FEE3FEE6FEE9FEEBFEEEFE26
:10943100F0FEF3FEF6FEF8FEFBFEFDFF00FF03FF6C
:1094410005FF08FF0BFF0DFF10FF12FF15FF18FFAF
:109451001AFF1DFF20FF22FF25FF27FF2AFF2DFFF7
:109461002FFF32FF35FF37FF3AFF3CFF3FFF42FF3F
:1094710044FF47FF49FF4CFF4FFF51FF54FF57FF88
:1094810059FF5CFF5EFF61FF64FF66FF69FF6CFFD0
:109491006EFF71FF73FF76FF79FF7BFF7EFF81FF18
:1094A10083FF86FF88FF8BFF8EFF90FF93FF96FF60
:1094B10098FF9BFF9DFFA0FFA3FFA5FFA8FFAAFFA9
:1094C100ADFFB0FFB2FFB5FFB8FFBAFFBDFFBFFFF1
:1094D100C2FFC5FFC7FFCAFFCDFFCFFFD2FFD4FF39
:0D94E100D7FFDAFFDCFFDFFFE2FFE4FFE76B
:1094EE00FFE9FFECFFEFFFF1FFF4FFF7FFF9FFFCE1
:1094FE00FFFE0000000300050008000A000D00102A
:10950E00001200150018001A001D001F0022002571
:10951E000027002A002D002F003200340037003AB9
:10952E00003C003F0042004400470049004C004F01
:10953E000051005400570059005C005E0061006449
:10954E0000660069006B006E007100730076007992
:10955E00007B007E0080008300860088008B008EDA
:10956E000090009300950098009B009D00A000A322
:10957E0000A500A800AA00AD00B000B200B500B86A
:10958E0000BA00BD00BF00C200C500C700CA00CCB3
:10959E0000CF00D200D400D700DA00DC00DF00E1FB
:1095AE0000E400E700E900EC00EF00F100F400F643
:1095BE0000F900FC00FE0101010401060109010B86
:1095CE00010E0111011301160118011B011E0120CC
:1095DE00012301260128012B012D01300133013514
:1095EE000138013B013D0140014201450148014A5C
:1095FE00014D0202040404040404040404040404DB
:10960E000404040404040404040406060606060600
:10961E0006060606060606060606060606060606DC
:10962E0006060606060606060606060606060606CC
:10963E0006060606060606080808080808080808AA
:10964E00080808080808080808080808080808088C
:10965E000808080A0A0A0A0A0A0A0A0A0A0A0A0A62
:10966E000A0A0A0A0A0A0A0A0A0A0A0A0A0A0A0A4C
:10967E000A0A0A0A0A0A0A0A0C0C0C0C0C0C0C0C2C
:10968E000C0C0C0C0C0C0C0C0C0C0C0C0C0C0C0C0C
:10969E000C0C0C0C0C0C0C0C0E0E0E0E0E0E0E0EEC
:1096AE000E0E0E0E0E0E0E0E0E0E0E0E0E0E0E0ECC
:1096BE000E0E0E0E0E0E0E0E0E0E0E0E0E0E0E0EBC
:1096CE00101010101010101010101010101010108C
:1096DE00101010101010101010101010101010127A
:1096EE001212121212121212121212121212151546
:1096FE0015180000000080005556400033342AAB88
:10970E00249320001C72199A1746155613B2124A4A
:10971E00111210000F100E390D7A0CCD0C310BA357
:10972E000B220AAB80008000800080008000800049
:10973E00800080008000800080008000800080001B
:10974E007AAB75C3713B6D096925658462225EF83B
:10975E005C0059365697541D51C74F914D794B7D2C
:10976E00499A47CE4618447742E9416C40003EA3E1
:10977E003D553C153AE139BA389E378C36853587DA
:10978E00349233A632C231E6311130432F7C2EBBD8
:10979E002E002D4B2C9B2BF12B4B2AAB2A0F29770E
:1097AE0028E4285427C9274126BD263C25BE25443A
:1097BE0024CD245823E72378230C22A3223C21D73F
:1097CE002174211420B6205A20001FA81F521EFDFE
:1097DE001EAB1E5A1E0A1DBD1D711D261CDD1C95BD
:1097EE001C4F1C0A1BC61B841B421B021AC31A8663
:1097FE001A491A0E19D3199A1961192A18F318BD94
:10980E0018891855182217EF17BE178D175D172ECA
:10981E00170016D216A51679164E162315F815CF63
:10982E0015A6157D1555152E150714E114BB1496A6
:10983E001472144E142A140713E413C213A0137FC8
:10984E00135E133E131E12FE12DF12C012A21284FA
:0D985E0012661249122C121011F411D811CB
:10986B00BC11A11186116C11511137111E1104106D
:10987B00EB10D310BA10A2108A1072105B104410A8
:10988B002D101610000FEA0FD40FBE0FA90F940F57
:10989B007F0F6A0F550F410F2D0F190F050EF20E8B
:1098AB00DE0ECB0EB80EA60E930E810E6E0E5C0E58
:1098BB004B0E390E1F0E050DEB0DD20DBA0DA10D72
:1098CB00890D710D5A0D430D2C0D160CFF0CEA0C66
:1098DB00D40CBF0CAA0C950C800C6C0C580C440CC3
:1098EB00310C1D0C0A0BF80BE50BD30BC10BAF0B9B
:1098FB009D0B8C0B7A0B690B580B480B370B270BFB
:10990B00170B070AF70AE70AD80AC90ABA0AAA0AFA
:10991B00AA0AAA0AAA0AAA0AAA0AAA0AAA0AAA0A9C
:10992B00AA0AAA0AAA0AAA0AAA0AAA0AAA0AAA0A8C
:10993B00AA0AAA0AAA0AAA0AAA0AAA0AAA0AAA0A7C
:01994B00AA71
:102D9A0030160B20260D301C0AD21DD22622D21E36
:042DAA001229F622D2
:10269C0090032F7403F0E4A3F0122E447E607F00AD
:1026AC007B017A03792F9002FFE4F0A304F0122946
:1026BC006B7E607F017B017A0379309002FFE4F03E
:1026CC00A304F012296B122B3D7E007F0A7D007B48
:1026DC00007A00795512152B755501E490032EF0F4
:1026EC0090032EE0FFC3941E502A75F00AEFA42429
:1026FC0002F582E5F03460AF82FE7B007A007955FA
:10270C009002FFE4F0A3740AF012296B90032EE000
:07271C0004F080CC022B3D0C
:102CF200906001E493F46009906000E493640360DF
:0A2D02000312269CE49002B2F022B6
:102A950090033E74FAF09002B2E0FFC3941E501EFC
:102AA500EF75F00AA42402F9746035F0FA7BFF781B
:0E2AB500557C007D007E007F0A1213F1C226C0
:012AC30022F0
:102A2C009002B2E0C3941E502B122E449002B2E0DE
:102A3C0075F00AA42402F582E5F03460AF82FE7BC7
:102A4C00007A0079559002FFE4F0A3740AF0122981
:052A5C006B122B3D226E
:062E7300122A2CC22622E7
:08193500900291EDF0A3EBF02C
:10193D00A3E004F0900296EFF0A3EBF0900291E09B
:10194D00FF900296E0FED39F40030219E975F00A5D
:10195D00EEA42402F582E5F03460AF82900298F097
:10196D00A3EFF0900297E075F00AA42402F582E54A
:10197D00F03460AF8290029AF0A3EFF0E4900294FD
:10198D00F0A3F090029AE475F0011214EFAFF0FE9F
:10199D00900298E0FCA3E0F5828C83E493FD12267F
:1019AD0010900299E004F07006900298E004F09017
:1019BD000295E004F07006900294E004F0C39002EA
:1019CD0095E0940A900294E0940040B7122B3D905C
:1019DD000296E004F0A3E004F00219499002B2E08F
:1019ED00FF900292E0D39F5009A3E0C39F400312E2
:0219FD002A9529
:0119FF0022C5
:0F1775009002A8EDF09002A7EFF09002A9EBF020
:101784009002AEEFF0A3EBF09002A8E0FF9002AE5F
:10179400E0D39F40030218F0A3E075F00AA42402EA
:1017A400F582E5F03460AF829002AAF0A3EFF0E492
:1017B4009002B0F0A3F09002B0E0FEA3E0FFC39467
:1017C4000AEE940050389002AAE0FCA3E0F5828C63
:1017D40083E493FD74B32FF582E43402F583EDF0D2
:1017E4009002ABE004F070069002AAE004F09002CC
:1017F400B1E004F070C09002B0E004F080B8900250
:10180400AEE075F00AA42402F582E5F03460AF82FC
:101814009002ACF0A3EFF09002AFE075F00AA424BC
:1018240002F582E5F03460AF829002AAF0A3EFF0F3
:10183400E49002B0F0A3F09002AAE475F00112144F
:10184400EFAFF0FE9002ACE0FCA3E0F5828C83E401
:1018540093FD1226109002ADE004F070069002ACE5
:10186400E004F09002B1E004F070069002B0E004ED
:10187400F0C39002B1E0940A9002B0E0940040B743
:101884009002AEE075F00AA42402F582E5F034601B
:10189400AF829002ACF0A3EFF0E49002B0F0A3F0BA
:1018A4009002B0E0FCA3E0FDC3940AEC9400502C39
:1018B4009002ACE475F0011214EFAFF0FE74B32D96
:1018C400F582E43402F583E0FD1226109002B1E0C3
:1018D40004F070CC9002B0E004F080C4122B3D9070
:1018E40002AEE004F0A3E004F002178C9002B2E030
:1018F400FF9002A9E0FED39F50209002A7E0FDA331
:10190400E0C39DFDE49400FCEE7A002DFDEA3CFC6E
:10191400C3ED9F7480F86C9850139002B2E0FF906E
:1019240002A7E0D39F5009A3E0C39F4003122A9566
:011934002290
:0B2354009002C7EFF0A3EDF0A3EBF048
:10235F00A2AFE433A3F0C2AF122E6D9002C8E0FE1D
:10236F009002C7E0FDEDFF9002CFEEF0A3EFF0E497
:10237F009002CBF09002C9E0FF9002CFE0FCA3E007
:10238F00FD7B017A0279B39002E9E4F0A3740AF0BD
:10239F00122BAB9002D0E0240AF09002CFE0340071
:1023AF00F09002CBE075F00AA42402F9746035F0C6
:1023BF00FAA374FFF0A3EAF0A3E9F0122E449002FF
:1023CF00CCA3E0FAA3E0AE02FF7B017A0279B390CF
:1023DF0002FFE4F0A3740AF012296B122B3D900256
:1023EF00CBE004F0E0C3941E408A900316E0FF1286
:0D23FF002DDA75CFE49002CAE024FF92AF02
:01240C0022AD
:0B2577009002DAEFF0A3EDF0A3EBF010
:10258200A2AFE433A3F0C2AF122E6D9002DBE0FEE5
:102592009002DAE0FDEDFF9002DFEEF0A3EFF0E44F
:1025A2009002DEF09002DEE0FFC3941E504C75F004
:1025B2000AEFA42402F582E5F03460AF82FE9002B5
:1025C200E1F0FAA3EFF0FB9002DCE0FF9002DFE023
:1025D200FCA3E0FDA9037BFF9002F1E4F0A3740ADF
:1025E200F0122CD89002E0E0240AF09002DFE034EE
:1025F20000F09002DEE004F080AA900316E0FF12E1
:0D2602002DDA75CFE49002DDE024FF92AFE9
:01260F0022A8
:102D3D00D209D208D207D206D205D204D203D202CA
:082D4D00D201E4F54FD220226F
:102D5500C209C208C207C206C205C204C203C20232
:082D6500C201E4F54FD2202267
:03000000020800F3
:03000300021A03DB
:03000B00021A06D0
:03001300021A09C5
:03001B00021A0CBA
:03002300021A0FAF
:03002B00021A12A4
:03003300021A1599
:03003B00021A188E
:03004300021A1B83
:03004B00021A1E78
:03005300021A216D
:03005B00021A2462
:03006300021A2757
:03006B00021A2A4C
:03007300021A2D41
:03007B00021A3036
:03008300021A332B
:03008B00021A3620
:03009300021A3915
:03009B00021A3C0A
:0300A300021A3FFF
:10080000787FE4F6D8FD9000007F007E20E4F0A31E
:0A081000DFFCDEFA75816202085574
:042C87008F828E8327
:102C8B00A2AF9227C2AF75B681758F03E4F0F58FB3
:072C9B0075B680A22792AF7D
:012CA200220F
:042C6A008F828E8344
:102C6E00A2AF9228C2AF758F0175B681EDF075B621
:082C7E0080E4F58FA22892AF5B
:012C8600222B
:10291F00900327EEF0A3EFF0A3ECF0A3EDF0EB4A5A
:10292F006039900327E0FEA3E0FFA3E0FCA3E0F5EE
:10293F00828C83E0FD122C6AEB1B70011A90032A24
:10294F00E004F07006900329E004F0900328E004FF
:0C295F00F070CB900327E004F080C3224E
:082E4400E4900000F0A3F0226D
:102B3D00900000E0FEA3E0FF122C87900000E0FE65
:102B4D00A3E0FF7C007D027B007A0212291FE49036
:062B5D000000F0A3F022CD
:0A261000A90590030DEEF0A3EFF012
:10261A00EE54FEFE900000E0FCA3E0FD7002EE6CBA
:10262A006057ED4C6003122B3D90030DE0FEEE5413
:10263A00FEFE7F00900000F0A3EFF090030FEEF093
:10264A00A3EFF0A37400F0A37402F07E0290030FCC
:10265A00E475F0011214EF85F082F583E493FD909E
:10266A000311E475F0011214EF85F082F583EDF0A1
:10267A00EF1F70011EEF4E70D490030DE0FCA3E033
:10268A00FDEC5401FC74022DF58274003CF583E9DB
:01269A00F04F
:01269B00221C
:10296B009002FAEEF0A3EFF0A3EBF0A3EAF0A3E9E9
:10297B00F09002FF74FFF5F01214EF45F060269013
:10298B0002FAE475F0011214EFAFF0FE9002FCE0D6
:10299B00FBA3E475F0011214EFA9F0FA121417FD62
:0629AB0012261080CC2270
:10081A0002089AE493A3F8E493A34003F68001F252
:10082A0008DFF48029E493A3F85407240CC8C333DF
:10083A00C4540F4420C8834004F456800146F6DFAE
:10084A00E4800B0102040810204080902C4CE47EC6
:10085A00019360BCA3FF543F30E509541FFEE493A3
:10086A00A360010ECF54C025E060A840B8E493A36A
:10087A00FAE493A3F8E493A3C8C582C8CAC583CA95
:10088A00F0A3C8C582C8CAC583CADFE9DEE780BE4D
:012C6900006A
:10132100E709F608DFFA8046E709F208DFFA803EAE
:1013310088828C83E709F0A3DFFA8032E309F6089B
:10134100DFFA8078E309F208DFFA807088828C8303
:10135100E309F0A3DFFA806489828A83E0A3F608B7
:10136100DFFA805889828A83E0A3F208DFFA804C91
:1013710080D280FA80C680D4806980F28033801068
:1013810080A680EA809A80A880DA80E280CA8033D1
:1013910089828A83ECFAE493A3C8C582C8CCC58349
:1013A100CCF0A3C8C582C8CCC583CCDFE9DEE78019
:1013B1000D89828A83E493A3F608DFF9ECFAA9F098
:1013C100EDFB2289828A83ECFAE0A3C8C582C8CCEE
:1013D100C583CCF0A3C8C582C8CCC583CCDFEADE07
:1013E100E880DB89828A83E493A3F208DFF980CC69
:1013F10088F0EF60010E4E60C388F0ED2402B40462
:101401000050B9F582EB2402B4040050AF23234508
:06141100822390137173A9
:10141700BB010689828A83E0225002E722BBFE02D3
:09142700E32289828A83E4932206
:10143000BB010CE58229F582E5833AF583E0225071
:1014400006E92582F8E622BBFE06E92582F8E222BB
:0D145000E58229F582E5833AF583E49322D5
:10145D00BB010689828A83F0225002F722BBFE016E
:02146D00F32268
:10146F00F8BB010DE58229F582E5833AF583E8F0B3
:10147F00225006E92582C8F622BBFE05E92582C85F
:02148F00F22247
:10149100EF8DF0A4A8F0CF8CF0A428CE8DF0A42E6F
:0214A100FE2229
:1014A300C2D5EC30E709B2D5E4C39DFDE49CFCEE64
:1014B30030E715B2D5E4C39FFFE49EFE121557C370
:1014C300E49DFDE49CFC800312155730D507C3E46B
:0614D3009FFFE49EFE22D3
:1014D900C5F0F8A3E028F0C5F0F8E582158270029E
:0614E9001583E038F0223B
:1014EF00A3F8E0C5F025F0F0E582158270021583B0
:0614FF00E0C838F0E8220D
:10150500D083D082F8E4937012740193700DA3A375
:1015150093F8740193F5828883E473740293686089
:06152500EFA3A3A380DF89
:10152B00EF4E6012EF60010EEDBB010B89828A83D7
:10153B00F0A3DFFCDEFA2289F05007F709DFFCA9E4
:0C154B00F022BBFEFCF309DFFCA9F0223B
:10155700BC000BBE0029EF8DF084FFADF022E4CC78
:10156700F875F008EF2FFFEE33FEEC33FCEE9DEC41
:10157700984005FCEE9DFE0FD5F0E9E4CEFD22ED87
:10158700F8F5F0EE8420D21CFEADF075F008EF2FD1
:10159700FFED33FD4007985006D5F0F222C398FDC2
:0515A7000FD5F0EA225F
:00000001FF
